:100000000C9472000C948D000C948D000C948D0057
:100010000C948D000C948D000C948D000C948D002C
:100020000C948D000C948D000C948D000C948D001C
:100030000C948D000C948D000C948D000C948D000C
:100040000C948D000C948D000C948D000C948D00FC
:100050000C948D000C948D000C948D000C948D00EC
:100060000C948D000C948D000C948D000C948D00DC
:100070000C948D000C948D000C948D000C948D00CC
:100080000C948D000C948D000C948D000C948D00BC
:100090000C948D000C948D000C948D000C948D00AC
:1000A0000C948D000C948D000C948D000C948D009C
:1000B0000C948D000C948D000C948D000C948D008C
:1000C0000C948D000C948D000C948D000C948D007C
:1000D0000C948D000C948D000C948D000C948D006C
:1000E0000C948D0011241FBECFEFD1E2DEBFCDBF37
:1000F00000E00CBF84B78093000214BE0FB6F894E2
:10010000A8958091600088618093600010926000E3
:100110000FBE0E94AA000C94E3000C94000090E033
:1001200080E081BB209108012E7F2093080120915F
:1001300008012160209308010196811521E09207B2
:1001400081F78FE39CE90197F1F700C0000090E090
:1001500080E00895F8948FEF80BB80910701816063
:10016000809307018091070182608093070111BA93
:10017000809108018160809308018091080182606C
:1001800080930801809108018D7F8093080185E3A9
:100190008A95F1F700008091080182608093080140
:1001A00085E38A95F1F70000789488E19EE00FB628
:1001B000F894A895809360000FBE90936000A89576
:0A01C0000E948F00FCCFF894FFCFDF
:00000001FF
